:040000008A01292820
:08000800F600F60E030EF700EE
:10001000040EF8000A0EF9008A010B1D13280B11BB
:1000200023208A110A12790E8A00780E8400770E36
:100030008300760E09004428772890289A28A4285F
:10004000E628FE28222943294C296F298A29AD292F
:10005000D52983160730831603139F008312831656
:10006000C0308100831225208A110A1224208A11AF
:100070000A1226208A110A1227208A110A12282021
:100080008A110A123628432883168316031306089A
:10009000C039860083120230FA0022208A110A1227
:1000A000333083120313AE001E208A110A1232303D
:1000B00083120313AE001E208A110A122C30831201
:1000C0000313AE001E208A110A1206308312031396
:1000D000AE001E208A110A120C3083120313AE00E8
:1000E0001E208A110A121C208A110A1208000130EF
:1000F00083120313AE001E208A110A120130FA0087
:1001000022208A110A12023083120313AE001E202D
:100110008A110A120130FA0022208A110A120800FC
:10012000831203132D08AF001030B0001F208A1176
:100130000A120800831203132E08AF000030B0002B
:100140001F208A110A120800831203132F08F100DE
:10015000F10CF10CF10C710C0F390F393004B100B6
:100160000608C0393104B100310886000130FA00B8
:1001700022208A110A128312031386160130FA0014
:1001800022208A110A128312031386122F080F39B4
:100190003004B1000608C0393104B10031088600CE
:1001A0000130FA0022208A110A12831203138616E4
:1001B0000130FA0022208A110A12831203138612D8
:1001C0000130FA0022208A110A1208008312031358
:1001D000B308031DEE288030B300F228C03083122C
:1001E0000313B300F101831203133308320703181A
:1001F000F10AAE001E208A110A120800F101303007
:10020000F2000830F300F401831203133408F50000
:100210000310F51B0314F40D0A30F402031812291D
:10022000F4070310F50DF30B08297408720703187F
:10023000F10A83120313AF001030B0001F208A119F
:100240000A120800DF30FB00000000000000000080
:10025000000000000000000000000000000000009E
:10026000000000000000000000000000000000008E
:100270000000000000000000FB0B29290000FA0B21
:10028000222900000800F001831203132408013E14
:100290000318F00AA40008000A3083120313240292
:1002A000031C6E29A401F1017F08013E0318F10A25
:1002B000FF00F1012608013E0318F10AA6000A30EA
:1002C0002602031C6E29A601F1012508013E031830
:1002D000F10AA500063025020318A50108008316BF
:1002E000831603130108F8390638810083120B08BE
:1002F000DF39A0388B008312A401FF01A601A501FC
:10030000A001FD01A801A701A301AC011B208A11D6
:100310000A1208003C307F02031CAC29F101831251
:1003200003132008013E0318F10AA000FF01F101A8
:100330007D08013E0318F10AFD000A307D02031C0E
:10034000AC29FD01F1012808013E0318F10AA800BB
:10035000063028020318A80108003C30831203135A
:100360002002031CD429F1012708013E0318F10AD9
:10037000A700A001F1012308013E0318F10AA30020
:100380000A302302031CCB29A301F1012C08013EF2
:100390000318F10AAC001830831203132702031C60
:1003A000D429A701A301AC01080000308312031374
:1003B000B2000030B30020208A110A128312031306
:1003C0002C08B40021208A110A1283120313230877
:1003D000B40021208A110A123A3083120313AD00AF
:1003E0001D208A110A12831203132808B400212049
:1003F0008A110A127D0883120313B40021208A1186
:100400000A122E3083120313AD001D208A110A1226
:10041000831203132508B40021208A110A128312C3
:0E04200003132608B40021208A110A120800D6
:04400E002A3FFC3F0A
:00000001FF
